S01D000062696E2F6F70656E626C745F73746D33326C3437362E7372656386
S31508000000008001202103000871030008710300081D
S31508000010710300087103000871030008000000005E
S315080000200000000000000000000000007103000846
S31508000030710300080000000071030008012200088F
S3150800004071030008710300087103000871030008B2
S3150800005071030008710300087103000871030008A2
S315080000607103000871030008710300087103000892
S315080000707103000871030008710300087103000882
S315080000807103000871030008710300087103000872
S315080000907103000871030008710300087103000862
S315080000A07103000871030008710300087103000852
S315080000B07103000871030008710300087103000842
S315080000C07103000871030008710300087103000832
S315080000D07103000871030008710300087103000822
S315080000E07103000871030008710300087103000812
S315080000F07103000871030008710300087103000802
S3150800010071030008710300087103000871030008F1
S3150800011071030008710300087103000871030008E1
S3150800012071030008710300087103000871030008D1
S3150800013071030008710300087103000871030008C1
S3150800014071030008710300087103000871030008B1
S3150800015071030008710300087103000871030008A1
S315080001607103000871030008710300087103000891
S3150800017071030008710300087103000800000000FD
S30D08000180710300087103000871
S3150800018810B5054C237833B9044B13B10448AFF3BB
S3150800019800800123237010BD3004002000000000F1
S315080001A80C220008084B10B51BB108490848AFF3DC
S315080001B800800848036803B910BD074B002BFBD01D
S315080001C8BDE81040184700BF0000000034040020AE
S315080001D80C220008300400200000000070B50F4EFD
S315080001E80F4D761BB61018BF002405D0013455F8F4
S315080001F8043B9847A642F9D10A4E0B4D761B02F0E6
S3150800020801F8B61018BF002406D0013455F8043B87
S315080002189847A642F9D170BD70BD00BFB022000844
S31508000228B0220008B8220008B0220008024B13B111
S31508000238024800F005B8704700000000550200089B
S31508000248002301461A46184600F014B838B5074D73
S31508000258074C2C1BA41005D0013C55F8043D9847BB
S31508000268002CF9D1BDE8384001F0D2BFBC220008FD
S31508000278B82200082DE9F047254C2568D5F84841E5
S315080002880646884692469946C4B360681F2817DC0E
S31508000298431C76B104EB80050122C5F888A0D4F87A
S315080002A8881182401143022EC4F88811C5F80891AE
S315080002B81ED00230636044F820800020BDE8F0872D
S315080002C8144B03B34FF4C870AFF300800446D0B19B
S315080002D8D5F84831002780E88800C5F848413846E7
S315080002E80123C4F88871C4F88C71002EE1D0D1E7CF
S315080002F8D4F88C110A43C4F88C21DAE705F5A674F4
S31508000308C5F84841C1E74FF0FF30BDE8F08700BFA0
S315080003182422000800000000DFF834D0002103E09A
S315080003280C4B5B58435004310B480C4B42189A4205
S31508000338F6D30B4A02E0002342F8043B094B9A42DB
S31508000348F9D300F06BF9FFF749FF00F00FF8FEE75D
S3150800035800800120BC22000800000020300400208C
S315080003683004002088090020FEE7000008B500F0E0
S3150800037887FC2C4A136823F0070343F00403136029
S31508000388136803F00703042B03D06A21264801F0F3
S315080003988BFB2649264B0A6822F4C06242F400728F
S315080003A80A601A6842F480721A601A461168204B65
S315080003B84805FBD559681F4A21F0F85141F0805184
S315080003C85960D9680A4042F4206242F00202DA60AB
S315080003D8DA6842F08072DA601A6842F080721A6047
S315080003E81968134A8901FBD5936843F00303936098
S315080003F891680F4B01F00C010C29F9D19A680E483F
S3150800040822F0F0029A609A6822F4E0629A609A6882
S3150800041822F460529A6000F0EFFE01F025FB01F025
S3150800042833FBFCE700200240282200080070004041
S31508000438001002408C80FFF900B4C404F0B53B4BA9
S315080004481A6E42F001021A661A6E8FB002F001029D
S315080004580792079A9A6D42F080529A659A6D02F049
S3150800046880520692069ADA6C42F00102DA64DA6C6D
S3150800047802F001020592059ADA6C42F00202DA6481
S31508000488DA6C02F002020492049ADA6C42F0040268
S31508000498DA64DA6C02F004020392039A9A6D42F45B
S315080004A800329A659A6D02F400320292029A9A6D9F
S315080004B842F000729A659B6D4FF0904703F00073FF
S315080004C800240193202508A901233846019A08958E
S315080004D809930A940B940C9400F096FABD620DEBF6
S315080004E805014FF400531248089302260325099478
S315080004F80C9400F089FA08A90C22072338460892B2
S315080005080D930B940C9409960A9500F07DFA4FF40E
S315080005184072092308A9074809960A950B940C946A
S3150800052808920D9300F070FA0FB0F0BD0010024063
S31508000538000800480004004810B54FF090442023EE
S31508000548A362134800F0C8F9124800F0C5F9204616
S3150800055800F0C2F9104B9A6D22F000729A659A6DEE
S3150800056822F400329A65DA6C22F00402DA64DA6C4C
S3150800057822F00202DA64DA6C22F00102DA649A6D71
S3150800058822F080529A651A6E22F001021A6610BD88
S3150800059800080048000400480010024008B500F0AA
S315080005A837F8024B1869C0F3403008BD0008004800
S315080005B8642000F003B800BF00F006B8014B1880A5
S315080005C8704700BF5004002010B50E4C01F0F8FD26
S315080005D8236898420ED30C4B1A7862B14FF09042B2
S315080005E8002020211870916201F0EAFD074B1B884C
S315080005F81844206010BD4FF0904201202021187041
S315080006089161F1E74C0400205204002050040020B0
S315080006184FF0904320229A62704700BF10B41149E0
S31508000628114BD1F8882042F47002C1F888201A685C
S31508000638002042F001021A6098601A6822F0A8524F
S3150800064822F410224FF480541A60DC601A684FF0BE
S31508000658006422F480221A6098618C605DF8044B65
S31508000668704700BF00ED00E000100240354B1B69DB
S315080006789A0704D5344A536843F001035360314B4B
S315080006881B691B0704D5304A536843F002035360B5
S315080006982C4B1B69D80604D52B4A536843F0040328
S315080006A85360284B1B69990604D5274A536843F0B3
S315080006B808035360234B1B695A0604D5224A536814
S315080006C843F0100353601F4B1B691B0604D51E4ACB
S315080006D8536843F0200353601A4B1B69D80504D5A1
S315080006E8194A536843F040035360164B1B6999052A
S315080006F804D5154A536843F080035360114B1B69A8
S315080007085A0404D5104A536843F4807353600D4B52
S315080007181B691B0404D50C4A536843F400735360D9
S31508000728084B9B69002B04DA074A536843F480632D
S315080007385360044B9A694CF2FA3142F000429A61C6
S31508000748196170470020024068090020064B5A695B
S31508000758002A01DB002070470449054A99609A6017
S315080007685869C00F704700BF00200240230167453B
S31508000778AB89EFCD034A536943F000435361002020
S31508000788704700BF0020024070B5054601F026FDF7
S315080007981F4C064601E06A1C30D123691C4ADB0354
S315080007A8F9D41369980725D41369190722D4136944
S315080007B8DB061FD413699E061CD413695D0619D473
S315080007C813691C0616D41369D80513D41369990531
S315080007D810D413695B040DD4136913F4004009D1C6
S315080007E89369002B06DB136913F001030DD0012367
S315080007F8136170BDFFF73AFF012070BD01F0EEFCEA
S31508000808801B8542C9D8032070BD184670BD00BF35
S31508000818002002402DE9F8432D4D2C78012C02D1F1
S315080008280220BDE8F8839846074601234CF2503063
S3150800083891460E462B70FFF7A7FF044610BB254ABC
S315080008486860136813F4806321D01368022123F4BF
S31508000858806313602977E7B91E4A536943F0010391
S3150800086853616FF00107C6F80090C6F804804CF289
S315080008785030FFF789FF174A53693B4004465361CE
S3150800088800F032FA00232B702046BDE8F8832B7750
S31508000898E1E77B1E012B05D94CF25030FFF774FFB0
S315080008A80446EDE70B494B6943F480234A464B61F6
S315080008B872B6B11A09F58074136853500432A24205
S315080008C8FAD162B6022FE7D16FF48027CFE700BFC7
S315080008D86809002000200240B0F1904F32D0424B00
S315080008E898423AD0414B984245D0414B984250D00D
S315080008F8404B98425BD0404B984266D03F4B984253
S3150800090804D03F4B98420FD00020704703F1F823D4
S3150800091803F580330120DA6A42F04002DA62DA6ABD
S3150800092822F04002DA62704703F1784303F5FA3396
S315080009380120DA6A42F08002DA62DA6A22F0800274
S31508000948DA6270472F4BDA6A42F00102DA62DA6A2B
S3150800095822F00102DA620120704703F1784303F5B1
S3150800096803330120DA6A42F00202DA62DA6A22F00E
S315080009780202DA62704703F1784303F5023301206D
S31508000988DA6A42F00402DA62DA6A22F00402DA6201
S31508000998704703F1784303F501330120DA6A42F018
S315080009A80802DA62DA6A22F00802DA62704703F1A4
S315080009B8784303F500330120DA6A42F01002DA6256
S315080009C8DA6A22F01002DA62704703F1784303F50F
S315080009D8FE330120DA6A42F02002DA62DA6A22F085
S315080009E82002DA62704700BF000400480008004881
S315080009F8000C004800100048001400480018004879
S31508000A08001C0048001002402DE9F0410A6892FAD5
S31508000A18A2F5B5FA85F532FA05F3D1F8048061D05E
S31508000A28012703264FF00F0E04E00A68013532FA4B
S31508000A3805F357D007FA05F31340F7D0026893FA77
S31508000A48A3FCBCFA8CFC93FAA3F4B4FA84F44FEA30
S31508000A584C0C640006FA0CFC08FA04F422EA0C02A8
S31508000A68224302604A68013A012A4AD9C26893FAB7
S31508000A78A3F4B4FA84F493FAA3FC640006FA04F41B
S31508000A8822EA0404BCFA8CFC0A694FEA4C0C02FAFE
S31508000A980CF22243C260D1F80480B8F1020FC4D11F
S31508000AA893FAA3F2B2FA82F2072A4FEA13243EDC33
S31508000AB8026A93FAA3F4B4FA84F493FAA3F3A400A3
S31508000AC80EFA04F422EA0404B3FA83F34A699B008B
S31508000AD802FA03F32343036291E80401013532FA63
S31508000AE805F3A7D108F1FF34012C07D8CB6841686C
S31508000AF803FB02F321EA02021A4342600120BDE819
S31508000B08F081826893FAA3F4B4FA84F493FAA3FCFE
S31508000B18640006FA04F422EA0404BCFA8CFC8A681F
S31508000B284FEA4C0C02FA0CF2224382609EE7D0F890
S31508000B3824C094FAA4F2B2FA82F294FAA4F39400BE
S31508000B48B3FA83F34A699B000EFA04F42CEA040400
S31508000B5802FA03F323434362D1F8048065E700BF2A
S31508000B68074AD1684FF6FF030B40000243F0BF63FC
S31508000B7800F4E06043F400330343D360704700BFD2
S31508000B8800ED00E030B4194BDB68C3F30223C3F168
S31508000B980705042D03F1040428BF0425062C18D9D3
S31508000BA8033B01249C40013C22400124AC40013C03
S31508000BB8214001FA03F3002842EA03020CDB00F19C
S31508000BC8604000F561401201D2B280F8002330BCBB
S31508000BD8704700221346E8E7054B00F00F0012019C
S31508000BE80344D2B21A7630BC704700BF00ED00E065
S31508000BF8FCEC00E00138B0F1807F0ED2084B10B447
S31508000C08084C58600022F020072184F823009A60CF
S31508000C18196010465DF8044B70470120704700BFFD
S31508000C2810E000E000ED00E010B5094B4FF0FF3288
S31508000C3800249A639C631A641C649A629C62DA624A
S31508000C48DC621A631C63FFF777FC204610BD00BFF9
S31508000C580010024010B5084B084A1B68A2FB03237C
S31508000C6804469809FFF7C6FF214600224FF0FF30D1
S31508000C78FFF788FF002010BD28040020D34D621016
S31508000C8808B5074A136843F4807313600320FFF70F
S31508000C9867FF0020FFF7DEFFFFF7D0FB002008BD3F
S31508000CA8002002400F4A5369C9074CBF23F4006362
S31508000CB843F4006353610B4B4FF4FF62596992FA88
S31508000CC8A2F2B2FA82F2904021F4FF621043586108
S31508000CD85A6942F002025A615A6942F480325A61E4
S31508000CE8704700BF00200240174B1A7F012A1CD004
S31508000CF81A7F032A19D01A7F1349022A05D00A7FB0
S31508000D08032A02D000221A777047104A116841F45C
S31508000D1880511160116821F480511160116841F4FD
S31508000D288061116000221A777047084A116841F4F1
S31508000D3800611160116821F400611160116841F4BD
S31508000D4800711160D7E700BF68090020002002403B
S31508000D582DE9F843414F3B78012B02D10220BDE823
S31508000D68F883044601254CF2503088463D70FFF753
S31508000D780BFD0646002842D1394B78601A6812F4EA
S31508000D88007F1A680CD022F400721A601A68500597
S31508000D9841D51A68032122F480621A60397702E07D
S31508000DA8510531D438772368012B36D04FF0FF33F5
S31508000DB8C8F80030A568E3682B449D421DD2DFF8C1
S31508000DC8A09005E0A268E36801351344AB4214D93C
S31508000DD861682846FFF766FF4CF25030FFF7D4FCE7
S31508000DE8D9F8143023F4FF6323F00203C9F8143042
S31508000DF80028E7D0C8F800500646FFF775FF002315
S31508000E083B703046BDE8F8831A68022122F48062EE
S31508000E181A603977C7E73D77C5E76368DA0704D5FF
S31508000E280F494A6942F004024A619B0704D50C4AED
S31508000E38536943F400435361094C636943F48033A7
S31508000E4863614CF25030FFF79FFC636923F4004353
S31508000E5823F0040306466361CFE700BF680900204C
S31508000E680020024010B41F4AD36803F00303022B7C
S31508000E782FD0032B2BD0136813F0080320D1116841
S31508000E88090756BFD2F894301268C3F30323164AE3
S31508000E9852F82340134BD968D868DB68C3F3416313
S31508000EA8C0F30622C1F30211013301315B00B4FB1A
S31508000EB8F1F05DF8044B02FB00F0B0FBF3F0704765
S31508000EC813681B0707D51368C3F30313DFE7074C33
S31508000ED8E0E7074CDEE7D2F894301B0903F0F00385
S31508000EE8D5E700BF001002404822000800127A0021
S31508000EF80024F4001C4B9B6803F00C030C2B08D841
S31508000F08DFE803F007070707190707071B07070797
S31508000F181D00154A136813F0080312D1116809074A
S31508000F2854BFD2F894301268104A58BFC3F3032343
S31508000F3852F8230070470E4870470E487047FFF767
S31508000F4891BF13681B0706D51368084AC3F303132A
S31508000F5852F823007047D2F89430044A1B0903F064
S31508000F68F00352F823007047001002404822000890
S31508000F780024F40000127A00032810B505D00C28BE
S31508000F8822D0302834D0002010BD314C314AD4F84C
S31508000F98883003F0030343F44033934250D0B3F147
S31508000FA8031F44D0013A93421ED0FFF7A3FFA36854
S31508000FB8A268294C2949C3F30313C2F3C222E35C86
S31508000FC88A5CD840D04010BD214C254AD4F88830D0
S31508000FD803F00C0343F44023934231D0B3F10C1FBA
S31508000FE825D0043A934213D1BDE81040FFF782BFD3
S31508000FF8174C1C4AD4F8883003F0300343F44013DE
S3150800100893421DD0B3F1301F11D0103A9342EBD05A
S31508001018FFF770FFA368A2680F4C1049C3F30313C0
S31508001028C2F30222E35C8A5CD840D04010BDD4F8EB
S31508001038903013F0020F0CBF00204FF4004010BD8B
S315080010482368094813F4806F08BF002010BD00BF45
S31508001058001002400200030030220008402200085F
S3150800106808000C00200030000024F400C02810B541
S3150800107824D0B0F5407F1FD1224C234AD4F88830B3
S3150800108803F4407343F04073934234D0B3F1032F0B
S3150800109828D0A2F58072934220D0FFF72BFFA368C9
S315080010A8A2681A4C1A49C3F30313C2F30222E35C73
S315080010B88A5CD840D04010BD002010BD114C154A96
S315080010C8D4F8883003F0C00343F44003934212D09F
S315080010D8B3F1C01F06D0403A9342DED1BDE81040AE
S315080010E8FFF708BFD4F8903013F0020F0CBF0020A2
S315080010F84FF4004010BD2368074813F4806F08BFF3
S31508001108002010BD0010024000020003302200082B
S31508001118402200088000C0000024F400F8B50368DF
S31508001128DB0728D404464F68C86826682C4B0D4642
S315080011380969AA69384301430A43334013432360BC
S315080011486268AB68274922F4405213436360A26871
S315080011586B6922F4407213438C42A36034D0224B45
S315080011689C4235D0214B9C4207D0214B9C4233D018
S31508001178204B9C4215D00020F8BD3020FFF7FCFE16
S315080011880028F8D02B68002BF5D0AA69B2F5004FCD
S315080011980CD000EB5300B0FBF3F080B2E0600120FE
S315080011A8F8BD4FF44070FFF761FFE9E75A084FF6B4
S315080011B8F07102EB4000B0FBF3F00140C0F34200C7
S315080011C80843E0600120F8BD0320FFF7D5FED7E7FE
S315080011D80C20FFF7D1FED3E7C020FFF747FFCFE77C
S315080011E8F369FFEF0038014000440040004800401A
S315080011F8004C004000500040014B1860704700BF83
S3150800120828040020704700BF002800F0838070B5C6
S3150800121890F820300446002B79D02268136823F00A
S315080012280203136000F0DAFF054604E000F0D6FF73
S31508001238401B0A2862D823685A689107F6D41A68A0
S3150800124842F001021A6000F0C9FF054604E000F002
S31508001258C5FF401B0A2851D823685A68D207F6D50D
S31508001268227E012A1A680CBF42F0800222F0800208
S315080012781A60637E2268012B13680CBF43F040038B
S3150800128823F040031360A37E2268012B13680CBF62
S3150800129843F0200323F020031360E37E2268012B22
S315080012A813680CBF23F0100343F010031360237F61
S315080012B82268012B13680CBF43F0080323F00803C0
S315080012C81360637F2268012B13680CBF43F004037D
S315080012D823F004031360A668E5682169626994E83F
S315080012E80900354329430A43013B134301210022D8
S315080012F8C361626284F82010104670BD636A0522CD
S3150800130843F40033636284F82020012070BDFFF798
S3150800131879FF82E70120704770B490F82030012BD6
S315080013280AD090F82030022B06D0436A43F480236B
S31508001338436270BC012070470368D3F8002242F064
S315080013480102C3F800224A69D3F81C02012404FAE8
S3150800135802F2D4432040C3F81C02C869B0B9D3F8CE
S315080013680C022040C3F80C024869CE688D884830BC
S3150800137845EA064543F8305048698D680E8848306E
S3150800138803EBC00046EA05454560C86901282AD026
S31508001398886910BBD3F804022040C3F80402086918
S315080013A8A8B9D3F814020440C3F81442096A0129F3
S315080013B804D1D3F81C120A43C3F81C22D3F8002216
S315080013C822F00102C3F80022002070BC7047D3F847
S315080013D814021043C3F81402E8E7D3F804021043CA
S315080013E8C3F80402DBE7D3F80C021043C3F80C026F
S315080013F848690E688D88483045EA064543F83050EE
S3150800140848698D688E89483003EBC00046EA054569
S315080014184560BDE738B590F82030012B05D0436AFA
S3150800142843F400234362012038BD0268022380F88A
S315080014382030136823F001031360044600F0CEFE3B
S31508001448054604E000F0CAFE401B0A2807D82368A8
S315080014585B6813F00103F5D16362184638BD636A01
S31508001468052243F40033636284F82020012038BD3E
S31508001478F0B590F82040012C83B00BD090F82040A6
S31508001488022C07D0436A43F48023436201210846A5
S3150800149803B0F0BD0468A5686F0102D4A5682E01DB
S315080014A840D5A4680125C4F30164A5401D608B686E
S315080014B84BBB0F68CB68066804F118054FEA051E8A
S315080014C843EA475346F80E3003680E6903EB0513DB
S315080014D85E600B7D012B2ED0230101685568CC1858
S315080014E80021C4F88C51046812681C44C4F8882181
S315080014F8026813440846D3F8802142F00102C3F86B
S31508001508802103B0F0BD06680196CE684F6804F1DD
S31508001518180533434FEA051E019E43EAC70346F8F2
S315080015280E30D1E7A568ED00BBD4436A43F400132F
S3150800153843620121ABE7016823011944D1F88441C4
S3150800154844F48074C1F88441C7E700BF90F8203096
S31508001558012B05D090F82030022B01D000207047C7
S3150800156803689B68890631EA030314BF0120002033
S31508001578704700BF70B4044690F8200001280AD0C6
S3150800158894F82000022806D0636A43F4802363622D
S31508001598012070BC7047256800295CD1E868860771
S315080015A869D001F11B000601AD5905F004059560DF
S315080015B8002D5BD02568AD59ED08556025680001F2
S315080015C80E012D58C5F34005D560256805446D6894
S315080015D805F00F051561256805446D68C5F30725E7
S315080015E89561256828444068000C50612068304495
S315080015F83246D0F8B801187020683044D0F8B801D7
S31508001608000A587020683044D0F8B801000C987061
S3150800161820683044D0F8B801000ED87020683044E5
S31508001628D0F8BC01187120683044D0F8BC01000A0B
S31508001638587120683044D0F8BC01000C98712068AD
S315080016480244D2F8BC21120EDA71D1B1012920D090
S31508001658002070BC70470129A3D128698007A0D14A
S31508001668636A43F400130846636292E72568AD592E
S315080016786D0D1560A2E7636A43F4001363620120DF
S3150800168887E72268D36843F02003D360084670BC0E
S3150800169870472268136943F020031361002078E72E
S315080016A8054B00221A709A6483F84320A3F844204D
S315080016B89A705A70704700BF54040020024B187875
S315080016C8003018BF0120704754040020024B00223E
S315080016D883F84320704700BF54040020F8B5037800
S315080016E8AE4CFF2B40D02278012A00D0F8BDC93B62
S315080016F80546352B00F23A81DFE813F0F300380186
S3150800170838017D00380138018C0069009400A10071
S3150800171838013801380138013801380138013801EB
S3150800172838013801380138013801380138013801DB
S3150800173838013801380138013801380138013801CB
S3150800174838013801380138013801380138013801BB
S31508001758B000C80024010B0138013801380113010B
S315080017683801D500DD00EA00002210210125E370C2
S31508001778217162706271257000F072F9A07100F02B
S315080017885FF9E07100F05CF90823D84020726572A9
S31508001798A572A4F8443000F049FA94F843307F4A11
S315080017A8012B05D0B2F9441000299FDD89B206E05D
S315080017B8FE2210230221E2702371A4F844100123A3
S315080017C884F843307648BDE8F84000F021B900F0BF
S315080017D847F96B78013898425DDDFF220123E270EC
S315080017E8A4F8443069786D4E002940F0CB8000F0A3
S315080017F827FA0028D1D1FE2131220223E17022716D
S31508001808A4F8443094F84330644A012BD0D0B2F88F
S315080018184410D4E700F020FAFF220123E270A4F866
S315080018284430EFE74168A06C5C4D00F003FA0028E5
S31508001838E1D0FF220123EA70A5F84430E2E7002543
S31508001848FF23E3702571657100F00AF90723A07173
S31508001858E57125726572A4F84430D3E7FF23E3706F
S315080018684368A26C3BB1D018002312F8011B0B443D
S315080018788242DBB2F9D1002201200821C4F80730D8
S3150800188820716271A271A4F84410BBE700F0E8F869
S315080018986B78984272DCFE2122220223E1702271BB
S315080018A8A4F84430AEE7FE2100220223E170227133
S315080018B8A4F84430A6E7FF2200236178E2700622DE
S315080018C82371A371E37123726171A4F8442099E71F
S315080018D80023FF21012223706370E170A4F84420D5
S315080018E890E7A76C2D4E00F0BBF86A1C411E3846D7
S315080018F800F09EF900283FF47EAFFF23F37000F04E
S31508001908AFF8B36C013803440122B364A6F844203F
S3150800191878E7FF23E3704368A3640123A4F84430F7
S3150800192870E7FF231F48E370072100230822A064F5
S3150800193823716371A37123726372A372E171A4F8A8
S3150800194844205FE700F08CF86A789042A3DDA16C22
S31508001958154800F0A3F9FF23E3706B78A26C1344CB
S31508001968A3646B780133A4F8443016E7FE212022D5
S315080019780223E1702271A4F8443043E76968A16438
S315080019886A78E5E7AA1CB06C00F052F900283FF41B
S3150800199832AF6B78B26C1344B364FEE65404002085
S315080019A857040020782200085804002010B5064C71
S315080019B8FFF776FE00F05EFB0123237000F0B8F807
S315080019C80023237010BD00BF2C04002008B50D485D
S315080019D800F0B0FB01280DD00A4800F0E1F801280C
S315080019E800D008BD084B074800221A70BDE8084011
S315080019F8FFF774BE044A034602481370FFF76EFEE3
S31508001A08EAE700BFA00400202C040020704700BFA6
S31508001A1870B50A4C2378012B0D46064608D01BB923
S31508001A28E9B2304600F09EF8BDE87040FFF74EBEB2
S31508001A38C9B200F057FB2378F1E700BF2C04002051
S31508001A48054B1B78013BDBB2022B9ABF034A32F8D7
S31508001A5813004020704700BF2C040020802200088D
S31508001A68FFF7EEBFFFF72ABE08B500F0F3F800F057
S31508001A7817F800F07DFB00F0D9F8FFF797FFBDE8E7
S31508001A88084000F031B800BF08B500F00BF800F0C0
S31508001A9889FBFFF79BFFBDE8084000F009B800BFBF
S31508001AA8FEF786BDFEF788BD08B5FFF7FBFFFCE71E
S31508001AB810B5FFF7D7FF012803D0094C2378012B67
S31508001AC800D010BD00F07CFB064B1B6803F5FA73C3
S31508001AD89842F6D300232370BDE8104000F0BCB83E
S31508001AE8E0040020E404002008B5054B01221A701A
S31508001AF800F066FB034B1860BDE80840FFF7D8BF3F
S31508001B08E0040020E404002038B5054600F058FB38
S31508001B18064CABB22385451D03E000F051FB854210
S31508001B2802D3E3691B06F8D538BD00BF0044004058
S31508001B3830B50B4C89B000230C224FF4614520467A
S31508001B4801A90293039304930693079301950592B3
S31508001B58FFF7E4FA236843F00103236009B030BDB0
S31508001B6800440040402938B50D46044611D8284691
S31508001B78ADB2FFF7C9FF5DB1013D14FA85F5013C21
S31508001B88FFF790FF14F8010FFFF7BEFFAC42F7D135
S31508001B9838BD75210148FFF787FFE8E7882200085E
S31508001BA870B51D4D2C7834B91C4BDA69920624D4C5
S31508001BB80024204670BD194AD46914F0200412D0AE
S31508001BC8174C18492378968CCA18013356700A7820
S31508001BD8DBB29A422370EBD1013100F05FF800239B
S31508001BE82B700124E5E700F0EBFA0F4B1B6864330A
S31508001BF89842DDD92C70204670BD9B8C094ADBB209
S31508001C081370002BD4D000F0DBFA074B044A18608F
S31508001C18012314702B70CCE7E90400200044004027
S31508001C28E8040020F0040020EC04002000F002B9C3
S31508001C3800F002B900F028B900F0DAB900F016BACF
S31508001C4808B500F0AFF900B908BDBDE8084000F0CE
S31508001C58F3B900BF00F0D2BA10B5FFF7EDFF00B927
S31508001C6810BDFEF79BFC0028FAD0FFF7CFFE00F060
S31508001C7893FAFEF7D9FFFFF7E1FF074B20F060401C
S31508001C8820F07F009860FFF7D9FF446800F0B8FA9B
S31508001C982346BDE81040184700ED00E072B170B55C
S31508001CA8561EB6B20D460644441E15F8013B04F8FE
S31508001CB8013FFFF7F7FEB442F7D170BD704700BF82
S31508001CC82DE9F0418046FEF741FD194B4FF40042D5
S31508001CD81A61002408E0D5E900239F4208BF964206
S31508001CE81AD1B4F5007F1DD008EB0403D3E90167C0
S31508001CF8D8F800502544FFF7D5FE32463B46294614
S31508001D080020FEF787FD08340028E4D00024FEF7F3
S31508001D1831FD2046BDE8F0810446FEF72BFD204636
S31508001D28BDE8F0810124FEF725FD2046BDE8F081CF
S31508001D380020024038B5104B98420D4619D00F4A74
S31508001D48914208D00446FFF7BBFF10B1C5F3080354
S31508001D5813B1002038BD1C462368AB4207D020467D
S31508001D68294640F8045B4FF40072FFF797FF2046B0
S31508001D7838BD034CEAE700BF3405002000280008F0
S31508001D88380700202DE9F8430C46016824F4FF7843
S31508001D981D464B1C0746164628F0010832D08845CA
S31508001DA806D038464146FFF7C5FF074638B30168E7
S31508001DB8641A3C44043408F5007807F1040905E078
S31508001DC816F8013B04F8013B013D15D0FFF76AFEFA
S31508001DD8C9EB0403B3F5007FF2D338464146FFF74B
S31508001DE8A9FF074658B100F104094C4616F8013B05
S31508001DF804F8013B013DE9D10120BDE8F88300203C
S31508001E08BDE8F8838146414649F8048B4FF40072C9
S31508001E184846FFF743FF3968C1E700BF0349044A44
S31508001E284FF0FF330B601360704700BF3807002078
S31508001E3834050020FFF7F2BF10B40F4CA04212D9A0
S31508001E484C1E0444B4F1016F0DD220F4FF730B4CF9
S31508001E5823F00103A3420B46014608D008485DF85B
S31508001E68044BFFF78FBF00205DF8044B7047054801
S31508001E785DF8044BFFF786BFFF270008002800080F
S31508001E883807002034050020F0B53F4B20F4FF67DB
S31508001E9827F007079F4287B05CD94B1E0344B3F166
S31508001EA8016F57D24518ED1BC5F30A03C5F3CF25AD
S31508001EB8002B5ED1FEF74AFC34494FF40040002255
S31508001EC80123086102920593002D55D0013DADB254
S31508001ED807F500632E4C2F4E03EBC52515E09A42ED
S31508001EE845D02D4B5202134003F100639F4234BF7D
S31508001EF80123022301A902A80393FEF729FF002854
S31508001F0840D107F50067AF4236D0FFF7CBFD2288E8
S31508001F184FF6FF739A4224D01F4B5202134003F11F
S31508001F2800639F4219D3FB1ADB0A1C4A04931368F9
S31508001F38228813F4807F4FF6FF73D0D09A4214D0C4
S31508001F48154B5202134003F100639F4234BF022324
S31508001F580123CFE7002007B0F0BD07F17843DB0A75
S31508001F68E3E7B742F9D90E4BDDE70D4BEDE70C4B26
S31508001F78BCE70135ADB29DE70124FEF7FBFB204619
S31508001F8807B0F0BD0024F8E7FF2700080020024044
S31508001F98E075FF1FFFFF070800FE1F00000001404D
S31508001FA800000808104B1A6801321AD0F0B5D3F8A1
S31508001FB804E09F68DE681D695C699969DA690B48F7
S31508001FC80EEB070333442B44234483B00B441344D2
S31508001FD802AA5B4242F8043D0421FFF72DFF03B02D
S31508001FE8F0BD0120704700BF340500208829000885
S31508001FF8F0B40D490D4B0E4A0F681B681568CC6876
S3150800200890680C4E3B4414312B4410320968126808
S31508002018234403440B4431681344CB420CBF0120C4
S315080020280020F0BC704700BF0028000804280008F4
S31508002038082800088829000808B50A4803680133EB
S3150800204802D0FFF73DFE58B107480368013305D0AB
S31508002058FFF736FE003018BF012008BD012008BD6D
S3150800206808BD00BF3405002038070020004870471F
S3150800207800280008F0B5194C194B23608BB00025C9
S315080020884FF480214FF4801214232046216162619F
S31508002098636025766576A576E57625776577A560FE
S315080020A8E5604FF6E077FFF7AFF8042601234CF60C
S315080020B8E04E0E226946204607930893CDF800E0BD
S315080020C80992059506950195049502970396FFF7D3
S315080020D823F92046FFF79EF90BB0F0BD3C0900200E
S315080020E80064004030B589B000240691024640F2E3
S315080020F8E17501AB02A90E48029504940594FFF709
S31508002108B7F908B109B030BD00F05AF800F1320441
S3150800211805E0FFF7C7FC00F053F88442F2D30199AB
S315080021280348FFF713FA0028F3D109B030BD00BFFA
S315080021383C09002000B589B0034601AA00210B48CE
S31508002148FFF718FA70B9019A40F267639A4202D003
S3150800215809B05DF804FB0398B0FA80F0400909B0A5
S315080021685DF804FB002009B05DF804FB3C09002073
S31508002178064B074910B40022064C1A6005205C6015
S315080021889A6018600A605DF8044B704710E000E032
S31508002198640900207F380100014B00221A60704745
S315080021A810E000E0044B1B68DB0303D5034A1368F9
S315080021B801331360704700BF10E000E0640900208F
S315080021C8044B1B6813F4803F034B18681CBF013087
S315080021D81860704710E000E064090020044B1B688B
S315080021E813F4803F034B18681CBF0130186070470A
S315080021F810E000E064090020704700BF72B6704717
S3150800220862B67047F8B500BFF8BC08BC9E4670476A
S31108002218F8B500BFF8BC08BC9E4670472D
S31508002224000000206D61696E2E6300000000000046
S315080022340000000001020304060708090000000064
S3150800224401020304A0860100400D0300801A06005B
S3150800225400350C0040420F0080841E0000093D0032
S3150800226400127A000024F40000366E010048E801E2
S31508002274006CDC024F70656E424C54000800000086
S31508002284000000002E2E2F2E2E2F2E2E2F536F7564
S315080022947263652F41524D434D345F53544D333267
S311080022A44C342F756172742E6300000024
S30D080022B035020008AD01000823
S309080022B88901000882
S315080022BC00000000EC02002054030020BC030020A0
S315080022CC00000000000000000000000000000000F4
S315080022DC00000000000000000000000000000000E4
S315080022EC00000000000000000000000000000000D4
S315080022FC00000000000000000000000000000000C4
S3150800230C00000000000000000000000000000000B3
S3150800231C00000000000000000000000000000000A3
S3150800232C0000000000000000000000000000000093
S3150800233C0000000000000000000000000000000083
S3150800234C0000000000000000000000000000000073
S3150800235C0000000000000000010000000000000062
S3150800236C0E33CDAB34126DE6ECDE05000B00000027
S3150800237C0000000000000000000000000000000043
S3150800238C0000000000000000000000000000000033
S3150800239C0000000000000000000000000000000023
S315080023AC0000000000000000000000000000000013
S315080026DC000000000000000000093D000400000096
S70508000321CE
